:101A4200EB88B3BAD87A7BA8FBFA3BC90212320000
:101A520000000000F1190BE91B329B6BFFFFFFFF37
:101A6200FFFFFEFEFDFCFCFBFAF9F8F7F6F5F3F2D8
:101A7200F0EFEDECEAE8E6E5E3E1DEDCDAD8D6D336
:101A8200D1CECCC9C7C4C2BFBCB9B7B4B1AEABA882
:101A9200A5A29F9C999693908C898683807D7A7764
:101AA20074706D6A6764615E5B5855524F4C49476A
:101AB20044413E3C393734322F2D2A282624221F16
:101AC2001D1B1A1816141311100E0D0B0A09080704
:101AD20006050404030202010101010101010101E1
:101AE2000101020203040405060708090A0B0D0E90
:101AF2001011131416181A1B1D1F222426282A2D12
:101B02002F323437393C3E414447494C4F525558A5
:101B12005B5E6164676A6D7074777A7D80838689A3
:101B22008C909396999C9FA2A5A8ABAEB1B4B7B97D
:101B3200BCBFC2C4C7C9CCCED1D3D6D8DADCDEE1B1
:101B4200E3E5E6E8EAECEDEFF0F2F3F5F6F7F8F9A3
:101B5200FAFBFCFCFDFEFEFFFFFFFFFF00000000A2
:101B62000000000000000000000000000000000073
:101B72000000000000000000000000000000000063
:101B82000000000000000000000000000000000053
:101B92000000000000000000000000000000000043
:101BA2000000000000000000000000000000000033
:101BB2000000000000000000000000000000000023
:101BC2000000000000000000000000000000000013
:101BD20000000000000000000000000001010101FF
:101BE20001010101010101010101010101010101E3
:101BF20001010101010101010101010101010101D3
:101C020001010101010101010101010101010101C2
:101C120001010101010101010101010101010101B2
:101C220001010101010101010101010101010101A2
:101C32000101010101010101010101010101010192
:101C42000101010101010101010101010101010182
:101C52000101010101010101010101013F800000B7
:101C6200404000004110000041D8000041A00000A7
:0C1C7200447A0000461C400047C35000AC
:1021C2008605A8FBFA0000008112FF41004501418B
:1021D2000095008210000082030100820C03E84493
:1021E200003D447A00008102004100960041005403
:1021F20001810F0148004C00000000000000004473
:102202000047000100014400410101010141005564
:10221200004100460041004B00810E0641003C0196
:09222200810B0181000081010023
:1024C200E4FDFCC3ED9FEC9E50070DBD00010C80A6
:0124D200F217
:0124D30022E6
:10244D00AB07AA06D3EB9400EA9400400E7F107EF2
:0C245D00271224C2EB1B70EC1A80E9224D
:102469007401A807088002C333D8FCF59DEF2480C6
:09247900F5BC7F017E000224C2C3
:10001E0043BC08E5BC30E4FB53BCE7AFBDEF75F065
:0D002E0004A4ADBE7C002DFFEC35F0FE22D9
:062316001508150815086A
:10231C00A80808E4F208F2A808F2A808E2C364804E
:10232C00948A501512001EA8080808E22FF218E231
:10233C003EF2A808E204F280E1A80808E2FE08E2F6
:01234C00FF91
:07234D000508050805082240
:0E250700E4F5C5F5C7F5C675C4FF75C3FF2220
:100003008FC4EEF5C375C78175C50175C65A75C62C
:07001300A5122507AFC22270
:102482008DC28FC4EEF5C375C78175C50275C65A74
:0624920075C6A502250736
:1024AE008FC4EEF5C375C78175C50375C65A75C65B
:0424BE00A502250747
:10222C00782A7401F2087400F2087456F2EF6028F0
:10223C00E4FFFE1224AEE4FCECFF7E00782AE2FB05
:10224C0008E2FA08E2F98C82758300120D84FD1203
:10225C0024820CECB40FE122E4FCECFF7E001200B3
:10226C0003782AE2FB08E2FA08E2F98C8275830013
:09227C00EF120DE50CECB40FE1CA
:012285002236
:092522007F067805E4F208DFFCF5
:01252B00228D
:1020CD009000BFE0F8A3E0F9A3E0FAA3E0FB120A49
:0420DD0066120CC8B3
:0520E1007837120EB675
:1020E600122522E4783BF2E47B0AFAF9F8C000787C
:1020F60037E2FC08E2FD08E2FE08E2FFD000122209
:10210600D274422BF582741A3AF583E493FF783B36
:10211600E22405F8EFF27837E2FC08E2FD08E2FE79
:1021260008E2FFE47B0AFAF9F81222D27837120E97
:10213600B67837E2FC08E2FD08E2FE08E2FFEC4D65
:0D2146004E4F6009783BE204F2E2B4069AC5
:012153002269
:101E2500FBE0FCA3E0FDA3E0FEA3E0FF120B6F784F
:0A1E3500317401F2780BE27832F20A
:051E3F00782D120EB623
:101E4400E47834F208F208F2FFFEFDFC782DE2FBA0
:101E540008E2F908E2FA08E2CBF8120C0C501A78FE
:101E6400367401F2782DE2FC08E2FD08E2FE08E295
:101E7400FF120C79782D120EB6E47833F2E4FFFEEB
:101E84007D7A7C44782DE2FB08E2F908E2FA08E264
:101E9400CBF8120C0C4021782DE2FC08E2FD08E29C
:101EA400FE08E2FFE4FBFA797A7844120B6F782D8E
:101EB400120EB67834E204F27833E204F2E2B403A8
:101EC400BCE47833F27831E2FF7833E2FEC3EF64A6
:101ED40080F8EE6480985042E4FFFE7D807C3F7879
:101EE4002DE2FB08E2F908E2FA08E2CBF8120C0C46
:101EF4005021782DE2FC08E2FD08E2FE08E2FFE44E
:101F0400FBFA797A7844120A66782D120EB6783480
:101F1400E214F27833E204F280ABE47833F2E4FFC3
:101F2400FE7D7A7C44782DE2FB08E2F908E2FA08A7
:101F3400E2CBF8120C0C5021782DE2FC08E2FD08EB
:101F4400E2FE08E2FFE4FBFA79207841120A66789F
:101F54002D120EB67835E204F27833E204F2E2B4DC
:101F640003BC7F007E407D1C7C46782DE2FB08E2AA
:101F7400F908E2FA08E2CBF8120975120CC812202B
:101F8400E17835E22405F8E22404F27832E26022B2
:101F94007834E2FF3395E0FE745A2FF582741A3ECA
:101FA400F583E4937805F27836E260067805E22456
:021FB40004F235
:011FB6002208
:1024980075D902E4F5F9F5E975FAC075EAC075DA97
:0624A80053D2BFD2AF22A7
:03003B0002228618
:10228600C0E0C083C082C0D075D000C000C006C008
:012296000740
:10229700C2D87810E2FF7802E22FFEEF901A5E9321
:1022A700F5FAAF06EF901B5E9324FF929208E2FEC9
:0C22B70008E2FF7811E22FF218E23EF27C
:0F22C300D007D006D000D0D0D082D083D0E03268
:10215400782BEEF208EFF218E2FC08E2FD780CECC2
:10216400F208EDF2E4120C8FE4FBFA79807847125E
:102174000A667B007A2479747847120B6F120CC8B4
:102184007803EEF208EFF2FDAC06E4120C8F7B004C
:102194007A2479747847120A66E4FBFA79807847DE
:1021A400120B6F90003D120EAAE47810F208F27838
:0E21B4002CE2700218E27003C2DE22D2DE229C
:10235400EF75F004120D49AFF0C3EF648094805020
:102364000474042FFFEF70037802F2EFB4010578D0
:10237400027440F2EFB4020578027480F2EFB40301
:0C23840005780274C0F2900096EFF02281
:09252C00900096E004FF02235424
:10240300EF7004C2A2C2A1EFB40104C2A2D2A1EF31
:10241300B40204D2A2C2A1EFB40304D2A2D2A19007
:052423000054EFF0225F
:1024E600900054E004FF75F004120D49AFF0022489
:0124F60003E2
:1023CB00D3EF6480948340027F03C3EF64809480D7
:1023DB005002E4FFEF7004C296C294EFB40104C242
:1023EB0096D294EFB40204D296C294EFB40304D203
:0823FB0096D294780FEFF22254
:1024F700780FE204FF75F004120D49AFF00223CB09
:10204300782AEFF2BFFF27E4F2780CE2FE08E2FF02
:1020530064644E7004782A04F2BE0308BFE805786E
:102063002A7402F2BE1E07BF8504E4782AF2782A96
:10207300E2700F7F64FE122154C295D2A0780E74D1
:102083000FF2782AE2B401107FE87E03122154C2D2
:1020930095C2A0780E7406F2782AE2B402107F8506
:1020A3007E1E122154D295C2A0780E7406F2782AAD
:1020B300E290003CF0758D2F758BABE4900046F0F9
:0A20C300900055F07810F208F222A8
:0B239000E0FEA3E0FFA3E0FCA3E0FDE3
:10239B00C3EE648094805007C3E49FFFE49EFEC3AA
:1023AB00EC648094805007C3E49DFDE49CFCD3ED6A
:1023BB009FEE6480F8EC6480984004AE04AF052275
:0A003E007814EBF208EAF208E9F288
:10004800900063E0FF3395E0FEA3E0FD3395E0FC0C
:10005800EF2DFFEE3C900097F0A3EFF0900059E0F1
:10006800FF3395E0FEA3E0FD3395E0FCEF2DFFEEB6
:100078003C900099F0A3EFF0A3120EC2000000001C
:100088009000A3120EC2000000007814E2FB08E200
:10009800FA08E2F9900006120E44FDACF0EC120CDE
:1000A8008FC004C005C006C0077814E2FB08E2FA56
:1000B80008E2F9900006120E44FDACF0EC120C8F29
:1000C800D003D002D001D000120A66C004C005C017
:1000D80006C0077814E2FB08E2FA08E2F990000487
:1000E800120E44FDACF0EC120C8FC004C005C00623
:1000F800C0077814E2FB08E2FA08E2F9900004125B
:100108000E44FDACF0EC120C8FD003D002D001D01D
:1001180000120A66D003D002D001D00012097590EF
:1001280000A7120EAA7814E2FB08E2FA08E2F99096
:100138000006120E44FDACF0EC120C8FC004C00592
:10014800C006C0077814E2FB08E2FA08E2F990005A
:1001580002120E44FDACF0EC120C8FD003D002D08A
:1001680001D000120A66C004C005C006C007781492
:10017800E2FB08E2FA08E2F9900004120E44FDAC32
:10018800F0EC120C8FC004C005C006C0077814E25A
:10019800FB08E2FA08E2F9120E19FDACF0EC120CB9
:1001A8008FD003D002D001D000120A66D003D0024B
:1001B800D001D000120975120C799000AB120EAA6A
:1001C8007814E2FB08E2FA08E2F9900002120E4401
:1001D800FDACF0EC120C8FC004C005C006C0077857
:1001E80014E2FB08E2FA08E2F9900004120E44FD5A
:1001F800ACF0EC120C8FD003D002D001D000120A60
:1002080066C004C005C006C0077814E2FB08E2FA1D
:1002180008E2F9900006120E44FDACF0EC120C8FC7
:10022800C004C005C006C0077814E2FB08E2FA085B
:10023800E2F9120E19FDACF0EC120C8FD003D002CB
:10024800D001D000120A66A804A905AA06AB07D0F7
:1002580007D006D005D004120971120C799000AFAE
:10026800120EAA9000A7E0F8A3E0F9A3E0FAA3E031
:10027800FBC000C001C002C0037817E2FB08E2FA25
:1002880008E2F9900002120D84FF3395E0FEEF7842
:1002980002C333CE33CED8F9245EF582741C3EF502
:1002A80083120E9AC000C001C002C0037817E2FB97
:1002B80008E2FA08E2F9120D6BFF3395E0FEEF78D9
:1002C80002C333CE33CED8F9245EF582741C3EF5D2
:1002D80083120E8AD003D002D001D000120B6FD047
:1002E80003D002D001D000120A669000A7120EAA0D
:1002F8009000A7E0FCA3E0FDA3E0FEA3E0FFC0049C
:10030800C005C006C007900054E0FF3395E0FE74B6
:100318005F2FF58274003EF583E0FC120C947B009D
:100328007A40791C7846120B6FE4FBFA7980783FA3
:10033800120975C004C005C006C007900054E0FF4C
:100348003395E0FEEF7802C333CE33CED8F9246E6E
:10035800F582741C3EF583120E9AD007D006D0059C
:10036800D004120A66A804A905AA06AB07D007D0CC
:1003780006D005D004120B6F9000A7120EAA7817AA
:10038800E2FB08E2FA08E2F9120D6BB4015E900094
:100398009BE0F8A3E0F9A3E0FAA3E0FBC000C001EA
:1003A800C002C003900059E0FC120C94D003D002A4
:1003B800D001D00012097590009B120EAA9000A3DC
:1003C800E0F8A3E0F9A3E0FAA3E0FBC000C001C095
:1003D80002C003900063E0FC120C94D003D002D05A
:1003E80001D0001209759000A3120EAA7817E2FB3B
:1003F80008E2FA08E2F9120D6BB4025E90009BE085
:10040800F8A3E0F9A3E0FAA3E0FBC000C001C00232
:10041800C00390005AE0FC120C94D003D002D00123
:10042800D00012097590009B120EAA9000A3E0F864
:10043800A3E0F9A3E0FAA3E0FBC000C001C002C03A
:1004480003900064E0FC120C94D003D002D001D0D9
:10045800001209759000A3120EAA7817E2FB08E2B1
:10046800FA08E2F9120D6BB4036690009BE0F8A35A
:10047800E0F9A3E0FAA3E0FBC000C001C002C0039A
:10048800900099E0FCA3E0FDEC120C8FD003D002A1
:10049800D001D00012097590009B120EAA9000A3FB
:1004A800E0F8A3E0F9A3E0FAA3E0FBC000C001C0B4
:1004B80002C003900097E0FCA3E0FDEC120C8FD083
:1004C80003D002D001D0001209759000A3120EAA21
:1004D8007817E2FB08E2FA08E2F9900002120D84AC
:1004E800B4016E90009BE0FCA3E0FDA3E0FEA3E056
:1004F800FFC004C005C006C007900059E0FC120CFC
:1005080094A804A905AA06AB07D007D006D005D041
:100518000412097190009B120EAA9000A3E0FCA39C
:10052800E0FDA3E0FEA3E0FFC004C005C006C007CD
:10053800900063E0FC120C94A804A905AA06AB0776
:10054800D007D006D005D0041209719000A3120E6E
:10055800AA7817E2FB08E2FA08E2F9900002120D05
:1005680084B4026E90009BE0FCA3E0FDA3E0FEA330
:10057800E0FFC004C005C006C00790005AE0FC12A6
:100588000C94A804A905AA06AB07D007D006D00585
:10059800D00412097190009B120EAA9000A3E0FCEF
:1005A800A3E0FDA3E0FEA3E0FFC004C005C006C0B1
:1005B80007900064E0FC120C94A804A905AA06ABF5
:1005C80007D007D006D005D0041209719000A312F5
:1005D8000EAA7817E2FB08E2FA08E2F99000021284
:1005E8000D84B4037690009BE0FCA3E0FDA3E0FE3D
:1005F800A3E0FFC004C005C006C007900099E0FC56
:10060800A3E0FDEC120C8FA804A905AA06AB07D03D
:1006180007D006D005D00412097190009B120EAACB
:100628009000A3E0FCA3E0FDA3E0FEA3E0FFC0046C
:10063800C005C006C007900097E0FCA3E0FDEC12DF
:100648000C8FA804A905AA06AB07D007D006D005C9
:10065800D0041209719000A3120EAA90009BE0FC2E
:10066800A3E0FDA3E0FEA3E0FFC004C005C006C0F0
:1006780007900054E0FF3395E0FE745B2FF5827419
:10068800003EF583E0FC120C94A804A905AA06AB69
:1006980007D007D006D005D00412097190009B122C
:1006A8000EAA90009BE0F8A3E0F9A3E0FAA3E0FB10
:1006B800C000C001C002C0037B007A2879F47845E5
:1006C80090003DE0FCA3E0FDA3E0FEA3E0FF120BD9
:1006D8006FE4FBFA797A7844120B6FD003D002D01A
:1006E80001D000120A6690009B120EAA90009BE0AF
:1006F800FCA3E0FDA3E0FEA3E0FFA804A905AA0669
:10070800FB120A66E4FBFAF97840120B6FA804A9F9
:1007180005AA06AB07E4FFFE7D807C3F12097190B5
:10072800009F120EAA9000A7E0F8A3E0F9A3E0FA50
:10073800A3E0FBC000C001C002C0037B007A40797F
:100748001C78469000A3E0FCA3E0FDA3E0FEA3E034
:10075800FF120B6FE4FBFA7980783F120975D0031A
:10076800D002D001D000120A669000A7120EAA90FB
:10077800009BE0FCA3E0FDA3E0FEA3E0FF9000AF38
:10078800E0F8A3E0F9A3E0FAA3E0FB120A66C004CC
:10079800C005C006C00790009FE0FCA3E0FDA3E0F1
:1007A800FEA3E0FF9000ABE0F8A3E0F9A3E0FAA312
:1007B800E0FB120A66D003D002D001D00012097102
:1007C8009000B3120EAA90009FE0FCA3E0FDA3E006
:1007D800FEA3E0FF9000AFE0F8A3E0F9A3E0FAA3DE
:1007E800E0FB120A66C004C005C006C00790009B63
:1007F800E0FCA3E0FDA3E0FEA3E0FF9000ABE0F87F
:10080800A3E0F9A3E0FAA3E0FB120A66D003D00242
:10081800D001D0001209759000AF120EAA9000B353
:10082800E0FCA3E0FDA3E0FEA3E0FF9000AB120E06
:10083800AA781A7401F2781AE2F9C36480948440A1
:1008480003020932E9FF3395E0FEEF7802C333CEA5
:1008580033CED8F92461F58274003EF583E0FCA319
:10086800E0FDA3E0FEA3E0FFC004C005C006C0078A
:10087800781AE2FF3395E0FEEF7802C333CE33CE29
:10088800D8F9FBAA062465F58274003AF583D007E7
:10089800D006D005D004120EAA74712BF58274000C
:1008A8003AF583E0FCA3E0FDA3E0FEA3E0FFC0046B
:1008B800C005C006C007781AE2FF3395E0FEEF785E
:1008C80002C333CE33CED8F9FBAA062475F5827459
:1008D800003AF583D007D006D005D004120EAA74CA
:1008E800812BF58274003AF583E0FCA3E0FDA3E0D8
:1008F800FEA3E0FFC004C005C006C007781AE2FFE7
:100908003395E0FEEF7802C333CE33CED8F9248591
:10091800F58274003EF583D007D006D005D00412C6
:100928000EAA781AE204F202083E9000A7E0FCA39F
:10093800E0FDA3E0FEA3E0FF900065120EAA900080
:10094800ABE0FCA3E0FDA3E0FEA3E0FF900075127E
:100958000EAA9000AFE0FCA3E0FDA3E0FEA3E0FF39
:06096800900085020EAABA
:03001B00021C7E46
:101C7E00C0E0C0F0C083C082C0D075D000C000C02C
:0D1C8E0001C002C003C004C005C006C007AD
:101C9B0090004BE06003021E0A900046E004F078CF
:101CAB000EE2FFE0C39F5003021E0AE4F0900055C2
:101CBB00E004F0E094044002E4F012231690003CA0
:101CCB00E0FD3395E0FC74562DF58274003CF583F2
:101CDB00E0FD3395E0FCC3EF9DFFEE9CFE9000967C
:101CEB00E0C3648094825006AC06AD078007C3E462
:101CFB009FFDE49EFC900055E0FB25E0244CF58213
:101D0B00E43400F583ECF0A3EDF0780FE2FD7441C1
:101D1B002BF582E43400F583EDF0C3EE6480948000
:101D2B0050047D0280027D00900055E0FC2447F5B5
:101D3B0082E43400F583E02DF074472CF582E43413
:101D4B0000F583E0FD75F004120D49ADF0EDF0ECFC
:101D5B0064016005EC6403707B900055E0B4010FE7
:101D6B00D297900050122390900043E07813F2909A
:101D7B000055E0B4030FC29790004C1223909000D3
:101D8B0041E07813F2D3EF9480EE648094A5400782
:101D9B007813E214F28036C3EF9440EE64809481A2
:101DAB0050087813E22403F28023C3EF94C0EE644F
:101DBB0080948350087813E22402F28010C3EF94CE
:101DCB0040EE6480948B50057813E204F27813E2B2
:101DDB00FF1223CB900055E00454032447F582E413
:101DEB003400F583E0FF12235478177401F2087462
:0F1DFB0000F2087441F27B017A00794C12003E2D
:101E0A00D007D006D005D004D003D002D001D0002C
:0B1E1A00D0D0D082D083D0F0D0E032D6
:0715D700782AEFF208EDF2A3
:1015DE009000B7120EC2000000009000BB120EC2A7
:1015EE00000000009000BF120EC200000000E47860
:1015FE002CF29000B7E0F8A3E0F9A3E0FAA3E0FB29
:10160E00C000C001C002C003782CE2FF3395E0FE9B
:10161E00EF7802C333CE33CED8F92465F582740049
:10162E003EF583E0FCA3E0FDA3E0FEA3E0FFE4FBB8
:10163E00FA79807840120B6FD003D002D001D0001F
:10164E001209759000B7120EAA9000BBE0F8A3E045
:10165E00F9A3E0FAA3E0FBC000C001C002C003780A
:10166E002CE2FF3395E0FEEF7802C333CE33CED8B3
:10167E00F92475F58274003EF583E0FCA3E0FDA32A
:10168E00E0FEA3E0FFE4FBFA79807840120B6FD006
:10169E0003D002D001D0001209759000BB120EAA21
:1016AE009000BFE0F8A3E0F9A3E0FAA3E0FBC000CE
:1016BE00C001C002C003782CE2FF3395E0FEEF7844
:1016CE0002C333CE33CED8F92485F58274003EF5AD
:1016DE0083E0FCA3E0FDA3E0FEA3E0FFE4FBFA79C8
:1016EE00807840120B6FD003D002D001D0001209C7
:1016FE00759000BF120EAA782CE204F2E264046028
:10170E00030216009000B7E0FCA3E0FDA3E0FEA3E9
:10171E00E0FFEC4D4E4F701012252278087473F2D4
:10172E0078067461F208F2227FDA7E0F7DC97C4062
:10173E0090003DE0F8A3E0F9A3E0FAA3E0FB120A63
:10174E00669000C7120EAA782BE2600302182F9043
:10175E0000B7E0FCA3E0FDA3E0FEA3E0FF9000C312
:10176E00120EAA782AE270139000C3E0F8A3E0F9F3
:10177E00A3E0FAA3E09000BF121E25782AE2B4017E
:10178E00139000C3E0F8A3E0F9A3E0FAA3E0900001
:10179E00BB121E25782AE264026003021946FFFE80
:1017AE00FDFC9000BFE0F8A3E0F9A3E0FAA3E0FB94
:1017BE00120C0C50359000BFE0F8A3E0F9A3E0FA4C
:1017CE00A3E0FBA3E0FCA3E0FDA3E0FEA3E0FF1279
:1017DE000B6F9000C7E0F8A3E0F9A3E0FAA3E0FBDB
:1017EE00120B6F783174040219439000C3E0F8A312
:1017FE00E0F9A3E0FAA3E0FB9000BFE0FCA3E0FD5C
:10180E00A3E0FEA3E0FF120B6F9000C7E0F8A3E089
:10181E00F9A3E0FAA3E0FB120B6F78317402021900
:10182E00439000BFE0FCA3E0FDA3E0FEA3E0FFA811
:10183E0004A905AA06FB120A66C004C005C006C0AC
:10184E00079000BBE0FCA3E0FDA3E0FEA3E0FFA831
:10185E0004A905AA06FB120A66D003D002D001D055
:10186E00001209759000B7E0F8A3E0F9A3E0FAA31F
:10187E00E0FB120B6F9000C3120EAA782AE27012D0
:10188E009000BFE0F8A3E0F9A3E0FAA3E0FBA312F7
:10189E001E26782AE2B401149000BBE0F8A3E0F90A
:1018AE00A3E0FAA3E0FB9000C3121E26782AE2649E
:1018BE00026003021946FFFEFDFC9000BFE0F8A394
:1018CE00E0F9A3E0FAA3E0FB120C0C50369000C333
:1018DE00E0F8A3E0F9A3E0FAA3E0FB9000BFE0FC80
:1018EE00A3E0FDA3E0FEA3E0FF120B6F9000C7E0A4
:1018FE00F8A3E0F9A3E0FAA3E0FB120B6F783174C2
:10190E000480329000BFE0F8A3E0F9A3E0FAA3E070
:10191E00FBA3E0FCA3E0FDA3E0FEA3E0FF120B6F30
:10192E009000C7E0F8A3E0F9A3E0FAA3E0FB120BE6
:10193E006F78317402121E38782AE2640360030253
:10194E001A419000BBE0FCA3E0FDA3E0FEA3E0FF84
:10195E00EC4D4E4F70087F0F7E27FDFC807590007A
:10196E00BBE0F8A3E0F9A3E0FAA3E0FBA3E0FCA33D
:10197E00E0FDA3E0FEA3E0FF120B6F122515900011
:10198E00BF120EAAE4FFFE7D7A7C449000BFE0F801
:10199E00A3E0F9A3E0FAA3E0FB120C0C400A7FE7E8
:1019AE007E037D007C00802BE4FFFE7DC87C429090
:1019BE0000BFE0F8A3E0F9A3E0FAA3E0FB120C0CE1
:1019CE0040149000BFE0FCA3E0FDA3E0FEA3E0FF07
:1019DE00120CC80220E1E4FFFE7D207C419000BF86
:1019EE00E0F8A3E0F9A3E0FAA3E0FB120C0C400E22
:1019FE00E4FFFE7D207C411220CD78068031E4FF8D
:101A0E00FE7D807C3F9000BFE0F8A3E0F9A3E0FAF2
:101A1E00A3E0FB120C0CE4FFFE400B7DC87C4212CF
:101A2E0020CD780780097D7A7C441220CD7808E29B
:031A3E002404F28B
:011A41002282
:10242800FF3395E0FE74422FF582741A3EF583E47B
:0224380093FF10
:10243A00EFF4F580D2A7C2A4C2A5C2A67F327E005D
:03244A0002244D1C
:100FC100E4781BF208F208F208F208F208F208F2DB
:100FD1000804F2E408F27F50FE12244DE4FF1222CD
:100FE1002CE4F588758912F58DF58BD28EC28CD2E1
:100FF100ABD2A9D2AFD2B9FF1224697596FF75920F
:10100100FC7591031224987F021223547F0112244C
:10101100031223CB7F011220437821E22401F2182D
:10102100E23400F2781EE204F25403F2C2A4C2A533
:10103100C2A6C2A7E2FF7002D2A7EFB40102D2A6F4
:10104100EFB40202D2A5EFB40302D2A474052FF8C3
:10105100E2F4F580E5B0F4781DF2E2600C18E2C329
:1010610094FF5005E204F28004E4781CF2E4781B5A
:10107100F2781DE2600AC313F2781BE204F280F1F8
:10108100781BE2781DF218E2B41407781F7432F26B
:101091008004E4781DF2781FE26007E214F2C2A333
:1010A1008002D2A3781DE2B4080BE4900045F0F26F
:1010B100782274FFF2900045E0FFC39401401AEFDB
:1010C100D394045014781DE2B407031224E6781D6A
:1010D100E2B406057FFF122043900045E070267FB1
:1010E100107E27FDFC1220E1781DE2FFC394014030
:1010F10010EFD39407500A900045EFF0E49000956B
:10110100F0E4781DF2900045E0640160030211E013
:1011110090004BF07822E2B4FF067401F2780BF2F2
:10112100781DE2B404157823E26006E4F27F7A8048
:101131000778237401F27FF112243A781DE2FFB49B
:1011410001137822E2780B7005E204F28003740146
:10115100F2E47822F2EFB402157822E2780BB401BE
:1011610005E204F280037401F278227401F2781D21
:10117100E2B403157822E2780BB40205E204F280AE
:10118100037401F278227402F2781DE2B405057845
:10119100227403F2780BE2FF75F002120D49AFF0F1
:1011A100780BEFF27822E2FF08E2FD1215D77823DF
:1011B100E2602C7820E25401FE08E2C39432EE94FE
:1011C10000501CE4781BF2781BE2FFC39404500F1B
:1011D10074052FF8E24404F2781BE204F280E890EF
:1011E1000045E0B40234900041E0FF3395E0FE7C1D
:1011F100007D64120E07900043E0FD3395E0FCEFA3
:101201002DFFEE3CCF2410CF3427FE3395E0FDFCBB
:101211001220E1E47808F27806F2900045E06403D8
:10122100704E90004B04F0781DE2B401091224F7CE
:10123100780FE2122428781DE2B4030EB297A29728
:10124100E433901A4293FF12243A781DE2B4040A5F
:1012510012252C900096E01224287821E2543F7048
:101261000F122316E4FCFD1220E17806E22404F2B9
:0B127100900045E0640760030215CD0B
:10127C00782704F208F208F2900095E0FF70167BD4
:10128C0001782404F2087400F2087456F2E4782809
:10129C00F2087402F2EFB4011578247401F20874A8
:1012AC0000F2087457F278287401F20804F2EFB4D3
:1012BC00021478247401F2087400F2087458F2785D
:1012CC00287402F208F2EFB4031578247401F208C2
:1012DC007400F208745BF278287402F2E408F2EFFE
:1012EC00B4041578247401F2087400F208745CF2EA
:1012FC0078287402F20814F2EFB4051478247401FF
:10130C00F2087400F208745DF278287402F208F2A4
:10131C00EFB4061578247401F2087400F208745EB8
:10132C00F278287402F20804F2EFB40715782474EA
:10133C0001F2087400F2087459F278287402F20869
:10134C0014F2EFB4081578247401F2087400F20852
:10135C00745AF278287402F20814F2EFB409177870
:10136C00247401F2087400F208745FF2087402F23B
:10137C000814F2E408F2EFB40A1678247401F208A7
:10138C007400F2087460F2087402F20814F208F2A5
:10139C00EFB40B1778247401F2087400F20874612E
:1013AC00F2087402F20814F20804F2EFB40C187884
:1013BC00247401F2087400F2087462F2087402F2E8
:1013CC000814F2087403F2EFB40D1678247401F2C9
:1013DC00087400F2087463F2087402F20814F2083C
:1013EC00F2EFB40E1678247401F2087400F208744B
:1013FC0064F2087402F20814F208F2781DE2B401E7
:10140C00127827E2FF7824E2FB08E2FA08E2F9EF0F
:10141C00120DB1781DE2B402177824E2FB08E2FA4F
:10142C0008E2F9120D6BFF08E2FEC3EF9E120DD31A
:10143C00781DE2B4030D7F0112222C90003CE0FFDA
:10144C00122043781DE2B4040E7824E2FB08E2FA81
:10145C0008E2F9E4120DD3781DE2640570359000B2
:10146C0095E07005740EF08006900095E014F0E4A1
:10147C007801F2900095E0FFC394095008EF901AA0
:10148C004293FF800B900095E0901A3C932404FF4C
:10149C0012243A781DE264067035900095E0B40E83
:1014AC0004E4F08006900095E004F0E47801F290FA
:1014BC000095E0FFC394095008EF901A4293FF8007
:1014CC000B900095E0901A3C932404FF12243A7878
:1014DC001DE2FFB407117801E204FE75F002120D53
:1014EC0049AEF07801EEF2EF6404704F7800E2043C
:1014FC00F26405704FF29000597410F0A37412F05E
:10150C00E4900063F0A3F0900056740FF0A37411F4
:10151C00F0A3740FF0E490005DF090005CF090008C
:10152C005BF090005E7414F0E4900062F090006147
:10153C00F0900060F090005FF08009781DE260048C
:10154C00E47800F27801E2603D90003CE0FE7828FF
:10155C00E2FF6E6003122043900054E0FE7829E213
:10156C00FF6E6003122403900095E0FFC3940340C8
:10157C000CEFD3940850067D017F0380047D017F1E
:10158C00011215D7803BE4780BF27824E2FB08E2D9
:10159C00FA08E2F9120D6BFF3395E0FE1224D4EE3B
:1015AC003395E0FDFC1220E17824E2FB08E2FA0816
:1015BC00E2F9120D6BC364809480500578087410A6
:0115CC00F22C
:0A15CD007FA07E0F1224C202101A44
:10096E00020D34E86480F8E933E83360110460F076
:10097E00ED33EC337009E8FCE9FDEAFEEBFF2204EF
:10098E0060DED3EB9FEA9EE99DE8C2E78CF0C2F7EA
:10099E0095F0400CE8CCF8E9CDF9EACEFAEBCFFBB6
:1009AE00120CFF85D0F05804700320D5B3E8047004
:1009BE00075002B2D5020D3E92D5EC0460F7E4CC9E
:1009CE00C0E0C398F8603B94186008400DD0E0FB7F
:1009DE00020D16E4FBFAC9FC8028E830E406E4C9EF
:1009EE00FBE4CAFCE830E305E4C9CACBFCE85407D3
:1009FE006010F8C3E913F9EA13FAEB13FBEC13FCDE
:100A0E00D8F130F52FC3E49CFCEF9BFFEE9AFEED80
:100A1E0099FDD0E0FBEF4E4D4C701222DB03020D20
:100A2E003BEC2CFCEF33FFEE33FEED33FDED30E708
:100A3E00EB020D16EF2BFFEE3AFEED39FDD0E0FB8B
:100A4E0050130BBB0003020D3EED13FDEE13FEEF34
:080A5E0013FFEC13FC020D165E
:100A6600EC4D6011E8497017ED33EC3304600DE48A
:100A7600FCFFFEFD22E933E8330470F8020D341260
:100A86000CFF58046009E4CC248150062850090262
:100A96000D3E284003020D3BC0E0EB4A7044B9808E
:100AA60006D0E0FB020D2AEF4E701CBD8008EBFF5E
:100AB600EAFEE9FD80EBE98DF0A4FEE5F0020B4FBE
:100AC600E9CDF9EAFEEBFFEF89F0A4FCE5F0CE896B
:100AD600F0A42EFFE435F0CD89F0A42DFEE435F028
:100AE6008067EF4E7005BD80D780C3EF8BF0A4AC56
:100AF600F0EE8BF0A42CFCE435F0F8EF8AF0A42C91
:100B0600E5F038FCE433CB8DF0A42CFCE5F03BF8A3
:100B1600EE8AF0A42CFCE5F038F8E433CF89F0A493
:100B26002CFCE5F038CF3400CE89F0A42FFFE5F099
:100B36003EFEE433C98DF0A42EFEE5F039CD8AF0F1
:100B4600A42FFFE5F03EFEE43DFD33D0E0FB500769
:100B56000BBB000F020D3EEC2CFCEF33FFEE33FE19
:060B6600ED33FD020D1647
:100B6C00020D3EEC5D046005E859047003020D347F
:100B7C00120CFF580460F6EC4860F2EC7004FDFEB9
:100B8C00FF22C860DB2481C85009C398600250065C
:100B9C00020D3B9850CAF582E9294B4A7005AB828D
:100BAC00020D2A75F0007C1A7880C3EF9BEE9AED4B
:100BBC0099400DC3EF9BFFEE9AFEED99FDE842F0D4
:100BCC00DC23ACF0D0E0FFD0E0FED0E0FDAB822027
:100BDC00E7101BEB60BAEC2CFCEF33FFEE33FEEDB1
:100BEC0033FD020D16E803F830E705C0F075F00090
:100BFC00EF2FFFEE33FEED33FD40B830E7C280AA95
:100C0C0074F8CC6480CCC86480C8F582046043C39B
:100C1C00EB9FF5F0EA9E42F0E99D42F0E89C45F02E
:100C2C0060305018E5825FFFE582F42B5582FB5053
:100C3C00210ABA001D09B90019088016E5825BFB70
:100C4C00E582F42F5582FF50090EBE00050DBD0044
:100C5C00010CC3EB9FF5F0EA9E42F0E99D42F0E8EF
:0D0C6C009C45F06007CC4820E701B3EC2266
:100C7900ED33EC33600A047003BD8004ECB2E7FC89
:010C89002248
:100C8A0075F020800E75F010800575F0087D007EE5
:100C9A00007F003392D530D503120E7CEC3340101E
:100CAA00EF33FFEE33FEED33FDEC33FCD5F0ED22EE
:0E0CBA00E5F0247EA2D513CC92E7CDCEFF222A
:100CC800EDD2E7CD33EC3392D524814006E4FFFE24
:100CD800FDFC22FCE4CFCECDCC24E0501174FF8083
:100CE800EDC3CC13CCCD13CDCE13CECF13CF047020
:070CF800F030D5DE020E7C96
:0D251500ED33EC3360065004EC6480FC22D2
:100CFF00E9D2E7C933E833F892D5EDD2E7CD33EC3B
:070D0F0033FC5002B2D522B3
:100D1600EC30E7100FBF000C0EBE00080DBD00043E
:100D26000BEB6014A2D5EB13FCED92E7FD2274FFEA
:100D3600FCFDFEFF22E480F8A2D574FF13FC7D8043
:030D4600E480EF57
:03000000021FB725
:0C1FB700787FE4F6D8FD758108021FFE5B
:100D4900C2D530F707B2D563F0FF05F030E70CB232
:100D5900D5F4048463F0FF05F080018430D502F4F2
:020D6900042262
:100D6B00BB010689828A83E0225002E722BBFE0286
:090D7B00E32289828A83E49322B9
:100D8400BB010CE58229F582E5833AF583E0225024
:100D940006E92582F8E622BBFE06E92582F8E2226E
:0D0DA400E58229F582E5833AF583E4932288
:100DB100BB010989828A83F8E028F022500327F7D2
:100DC10022BBFE05F8E328F3228A838982F8E493A3
:020DD1002822D6
:100DD300BB010689828A83F0225002F722BBFE01FF
:020DE300F322F9
:100DE500F8BB010DE58229F582E5833AF583E8F044
:100DF500225006E92582C8F622BBFE05E92582C8F0
:020E0500F222D7
:100E0700EF8DF0A4A8F0CF8CF0A428CE8DF0A42EFF
:020E1700FE22B9
:100E1900BB010A89828A83E0F5F0A3E022500687A4
:100E2900F009E71922BBFE07E3F5F009E319228966
:0B0E3900828A83E493F5F07401932299
:100E4400BB0110E58229F582E5833AF583E0F5F0EC
:100E5400A3E0225009E92582F886F008E622BBFEC9
:100E64000AE92582F8E2F5F008E222E5832AF5830F
:080E7400E993F5F0A3E99322D4
:1022D200C2D5E830E70FB2D5E4C39BFBE49AFAE437
:1022E20099F9E498F8EC30E717B2D5122308120FE7
:1022F2002FE4C39BFBE49AFAE499F9E498F880038B
:10230200120F2F30D50DE4C39FFFE49EFEE49DFD26
:04231200E49CFC2229
:0E0E7C00C3E49FFFE49EFEE49DFDE49CFC2287
:100E8A00E493FC740193FD740293FE740393FF22AE
:100E9A00E493F8740193F9740293FA740393FB22AE
:0C0EAA00ECF0A3EDF0A3EEF0A3EFF022BB
:0C0EB600ECF208EDF208EEF208EFF22278
:100EC200A8828583F0D083D082120ED9120ED91255
:100ED2000ED9120ED9E473E493A3C583C5F0C5837A
:100EE200C8C582C8F0A3C583C5F0C583C8C582C87A
:010EF20022DD
:1024D400C3EE6480948040028007C3E49FFFE49EBF
:0224E400FE22D6
:101FC300020FC1E493A3F8E493A34003F68001F264
:101FD30008DFF48029E493A3F85407240CC8C3331F
:101FE300C4540F4420C8834004F456800146F6DFEE
:101FF300E4800B01020408102040809021C2E47E9B
:10200300019360BCA3FF543F30E509541FFEE493E2
:10201300A360010ECF54C025E060A840B8E493A3A9
:10202300FAE493A3F8E493A3C8C582C8CAC583CAD4
:10203300F0A3C8C582C8CAC583CADFE9DEE780BE8C
:01222B0000B2
:100EF30075F008758200EF2FFFEE33FECD33CDCCB6
:100F030033CCC58233C5829BED9AEC99E582984038
:100F13000CF582EE9BFEED9AFDEC99FC0FD5F0D615
:100F2300E4CEFBE4CDFAE4CCF9A88222B800C1B93F
:100F33000059BA002DEC8BF084CFCECDFCE5F0CB7D
:100F4300F97818EF2FFFEE33FEED33FDEC33FCEBB6
:100F530033FB10D703994004EB99FB0FD8E5E4F971
:100F6300FA227818EF2FFFEE33FEED33FDEC33FC5E
:100F7300C933C910D7059BE99A4007EC9BFCE99A52
:100F8300F90FD8E0E4C9FAE4CCFB2275F010EF2F97
:100F9300FFEE33FEED33FDCC33CCC833C810D70797
:100FA3009BEC9AE899400AED9BFDEC9AFCE899F8D2
:0E0FB3000FD5F0DAE4CDFBE4CCFAE4C8F92265
:00000001FF
